:03200000022100BA
:03202B00022FF58C
:1021000075BF0143B70843B70453B6F743B6047924
:1021100000780AD9FED8FC785643B602D8FEE5B658
:1021200030E0F475BB9853B70F43B7A053B7FB43E8
:10213000B7027864D8FEE5B730E0DC53B7F775BF77
:102140000078FFE4F6D8FD90F0007F007E06E4F012
:10215000A3DFFCDEFA75819F0221960221DBE49366
:10216000A3F8E493A34003F68001F208DFF480298A
:10217000E493A3F85407240CC8C333C4540F442079
:10218000C8834004F456800146F6DFE4800B010268
:10219000040810204080902A34E47E019360BCA3A0
:1021A000FF543F30E509541FFEE493A360010ECFB6
:1021B00054C025E060A840B8E493A3FAE493A3F8E0
:1021C000E493A3C8C582C8CAC583CAF0A3C8C582A0
:1021D000C8CAC583CADFE9DEE780BE122B5FE4F51B
:1021E000BF7581C0D280D2947D02FF1240617B0115
:1021F0007AF079EE123BF990F116EEF0A3EFF07B56
:10220000017AF079541235B51230FC122E4A12427E
:102210009B122EC480F27C01122D997F027E002237
:10222000022568E86480F8E933E83360110460F05F
:10223000ED33EC337009E8FCE9FDEAFEEBFF220424
:1022400060DED3EB9FEA9EE99DE8C2E78CF0C2F71F
:1022500095F0400CE8CCF8E9CDF9EACEFAEBCFFBEB
:1022600012253385D0F05804700320D5B3E80470EC
:10227000075002B2D502257292D5EC0460F7E4CC87
:10228000C0E0C398F8603B94186008400DD0E0FBB4
:1022900002254AE4FBFAC9FC8028E830E406E4C9D8
:1022A000FBE4CAFCE830E305E4C9CACBFCE8540708
:1022B0006010F8C3E913F9EA13FAEB13FBEC13FC13
:1022C000D8F130F52FC3E49CFCEF9BFFEE9AFEEDB6
:1022D00099FDD0E0FBEF4E4D4C701222DB0302253E
:1022E0006FEC2CFCEF33FFEE33FEED33FDED30E70A
:1022F000EB02254AEF2BFFEE3AFEED39FDD0E0FB75
:1023000050130BBB0003022572ED13FDEE13FEEF1D
:1023100013FFEC13FC02254AEC4D6011E8497017DD
:10232000ED33EC3304600DE4FCFFFEFD22E933E8FD
:10233000330470F802256812253358046009E4CC90
:102340002481500628500902257228400302256F77
:10235000C0E0EB4A7044B98006D0E0FB02255EEF96
:102360004E701CBD8008EBFFEAFEE9FD80EBE98DB5
:10237000F0A4FEE5F0022401E9CDF9EAFEEBFFEF5F
:1023800089F0A4FCE5F0CE89F0A42EFFE435F0CD71
:1023900089F0A42DFEE435F08067EF4E7005BD8016
:1023A000D780C3EF8BF0A4ACF0EE8BF0A42CFCE450
:1023B00035F0F8EF8AF0A42CE5F038FCE433CB8D4F
:1023C000F0A42CFCE5F03BF8EE8AF0A42CFCE5F040
:1023D00038F8E433CF89F0A42CFCE5F038CF340092
:1023E000CE89F0A42FFFE5F03EFEE433C98DF0A4C2
:1023F0002EFEE5F039CD8AF0A42FFFE5F03EFEE495
:102400003DFD33D0E0FB50070BBB000F022572EC03
:102410002CFCEF33FFEE33FEED33FD02254A02259F
:1024200072EC5D046005E85904700302256812250A
:1024300033580460F6EC4860F2EC7004FDFEFF22B5
:10244000C860DB2481C85009C39860025006022589
:102450006F9850CAF582E9294B4A7005AB82022574
:102460005E75F0007C1A7880C3EF9BEE9AED994080
:102470000DC3EF9BFFEE9AFEED99FDE842F0DC23E1
:10248000ACF0D0E0FFD0E0FED0E0FDAB8220E71062
:102490001BEB60BAEC2CFCEF33FFEE33FEED33FDAB
:1024A00002254AE803F830E705C0F075F000EF2F89
:1024B000FFEE33FEED33FD40B830E7C280AA75F081
:1024C00020800E75F010800575F0087D007E007F7D
:1024D000003392D530D5031226B4EC334010EF33DD
:1024E000FFEE33FEED33FDEC33FCD5F0ED22E5F0ED
:1024F000247EA2D513CC92E7CDCEFF22EDD2E7CD3C
:1025000033EC3392D524814006E4FFFEFDFC22FC2F
:10251000E4CFCECDCC24E0501174FF80EDC3CC13BA
:10252000CCCD13CDCE13CECF13CF0470F030D5DE8B
:102530000226B4E9D2E7C933E833F892D5EDD2E701
:10254000CD33EC33FC5002B2D522EC30E7100FBF94
:10255000000C0EBE00080DBD00040BEB6014A2D5EC
:10256000EB13FCED92E7FD2274FFFCFDFEFF22E47D
:1025700080F8A2D574FF13FC7D80E480EFBB0106D8
:1025800089828A83E0225002E722BBFE02E322898D
:10259000828A83E49322BB010CE58229F582E583DC
:1025A0003AF583E0225006E92582F8E622BBFE06D2
:1025B000E92582F8E222E58229F582E5833AF5836E
:1025C000E49322BB010FF8E58229F582E5833AF511
:1025D00083E028F0225009C58229F8E58226F622F8
:1025E000BBFE09C58229F8E22582F222F8EA25839A
:1025F000F583E9932822BB010689828A83F0225061
:1026000002F722BBFE01F322F8BB010DE58229F59A
:1026100082E5833AF583E8F0225006E92582C8F680
:1026200022BBFE05E92582C8F222BC000BBE0029B0
:10263000EF8DF084FFADF022E4CCF875F008EF2FB9
:10264000FFEE33FEEC33FCEE9DEC984005FCEE9D76
:10265000FE0FD5F0E9E4CEFD22EDF8F5F0EE842092
:10266000D21CFEADF075F008EF2FFFED33FD4007F3
:10267000985006D5F0F222C398FD0FD5F0EA22A3B8
:10268000F8E0C5F025F0F0E582158270021583E0D0
:10269000C838F0E822BB010A89828A83F0E5F0A3FA
:1026A000F0225006F709A7F01922BBFE06F3E5F069
:1026B00009F31922C3E49FFFE49EFEE49DFDE49C20
:1026C000FC22EB9FF5F0EA9E42F0E99D42F0EC64BB
:1026D00080C864809845F022EB9FF5F0EA9E42F0B6
:1026E000E99D42F0E89C45F022E8600FECC313FC42
:1026F000ED13FDEE13FEEF13FFD8F122E8600FEFAC
:10270000C333FFEE33FEED33FDEC33FCD8F122BBD7
:10271000010789828A83022A0C5005E9F8022A00FF
:10272000BBFE05E9F8022A1889828A83022A24EC72
:10273000F0A3EDF0A3EEF0A3EFF022A8828583F0E2
:10274000D083D082122752122752122752122752B8
:10275000E473E493A3C583C5F0C583C8C582C8F0FC
:10276000A3C583C5F0C583C8C582C822E3F5F009B7
:10277000E208B5F06BDFF58067E3F5F009E608B530
:10278000F05EDFF5805A87F009E608B5F052DFF613
:10279000804E87F009E208B5F046DFF68042888275
:1027A0008C8387F009E0A3B5F036DFF680328882AB
:1027B0008C8387F009E493A3B5F025DFF5802188A9
:1027C000828C83E3F5F009E0A3B5F014DFF5801007
:1027D00088828C83E3F5F009E493A3B5F002DFF47B
:1027E000022897808780E9809080D4803C80158083
:1027F0006C807C809D80B7808D80A3804F807280AC
:102800003A0228A389828A8363A20188828C836327
:10281000A201E493F5F0A363A201E493A363A201F0
:10282000B5F074DFEDDEEB806E89828A83E493F588
:10283000F0A3E208B5F060DFF4805C89828A83E06F
:10284000F5F0A3E608B5F04FDFF5804B89828A8367
:10285000E0F5F0A3E208B5F03EDFF5803A89828A20
:1028600083E493F5F0A3E608B5F02CDFF48028802C
:1028700002805389828A8363A20188828C8363A247
:1028800001E493F5F0A363A201E0A363A201B5F014
:1028900006DFEEDEEC80007FFFB5F0020F22400283
:1028A0007F012289828A8363A20188828C8363A24A
:1028B00001E0F5F0A363A201E0A363A201B5F0D7A4
:1028C000DFEFDEED80D189828A8363A20188828C6A
:1028D0008363A201E0F5F0A363A201E493A363A2E2
:1028E00001B5F0B3DFEEDEEC80AD88F0EF60010EF5
:1028F0004E60AFED2402B40400509CF582EB24023C
:10290000B40400509223234582239027E373E70900
:10291000F608DFFA8046E709F208DFFA803E88828F
:102920008C83E709F0A3DFFA8032E309F608DFFAC7
:102930008076E309F208DFFA806E88828C83E309EF
:10294000F0A3DFFA806289828A83E0A3F608DFFAC7
:10295000805689828A83E0A3F208DFFA804A80D217
:1029600080FA80C680D4806580F28031801080A695
:1029700080EA809A80A880DA80E280CA80318982E9
:102980008A8363A20188828C8363A201E493A36398
:10299000A201F0A363A201DFF3DEF1800B89828A3A
:1029A00083E493A3F608DFF9ECFAA9F0EDFB2289A2
:1029B000828A8363A20188828C8363A201E0A3637D
:1029C000A201F0A363A201DFF4DEF280DB89828A38
:1029D00083E493A3F208DFF980CE88F0EF60010E64
:1029E0004E60C588F0ED2402B4040050BBF582EBC4
:1029F0002402B4040050B1232345822390295E733E
:102A0000E6FC08E6FD08E6FE08E6FF22E0FCA3E09F
:102A1000FDA3E0FEA3E0FF22E2FC08E2FD08E2FEE7
:102A200008E2FF22E493FC740193FD740293FE74A8
:102A30000393FF2258F00000000000000000000097
:102A40000000000000000000000000000000004442
:102A5000F0470000000042F03C0000C100C101420C
:102A6000F03A03E848F03E00000000000000004893
:102A7000F04B000000000000000048F021000000C2
:102A8000000000000048F0540001010000000000B8
:102A900048F029000000000000000050F06D000028
:102AA000000000000000000000000000000050F0E6
:102AB0005D000000000000000000000000000000B9
:102AC0000048F019000000000000000048F032004B
:102AD0000000000000000041F0310050F07E0000D6
:102AE000000000000000000000000000000041F0B5
:102AF000460041F0180041F07D00C102C10341F0E1
:102B00005C0041F0530048F0E600000000000000C7
:102B100000008E198F188C1C8D1BE4F51DF51EF519
:102B20001FC0D0C0E0C0F043D01812DFF94008D079
:102B3000F0D0E0D0D0D322D0F0D0E0D0D0C3228FDC
:102B400018C0D0C0E0C0F043D01812DFF64008D063
:102B5000F0D0E0D0D0D322D0F0D0E0D0D0C32275D6
:102B6000BF0175BA10E4F5BFB1A9F1E3D11F123F5F
:102B7000EF7181F1D0E4F5B8F5B9F5F8F5F9D2AF18
:102B80002275DA0075D97175DC01E5DC30E005539A
:102B9000D8FE80F675DA0075D98075DB4975D815D1
:102BA000E5D820E1FB75D804D116E5D820E1FBD1AA
:102BB00016E5D820E1FB75DB4B75DC3A75D835E5B9
:102BC000D820E1FB75DD6075D845E5D820E1FBE450
:102BD000F5DBF5DCF5DD75D871E5D820E1FB75DABC
:102BE0000075D9C075DB4175D815E5D820E1FB75B6
:102BF000B202439002439102E4F5B2439102F5DA46
:102C000075D9717F02FE7D081222167D05122216EB
:102C10007D061222167D071222167D091222167DCC
:102C20000A1222167D0B1222167D0C1222167D0D21
:102C30007C01B19975DA0475D92FD10FB1917F0359
:102C40007E007D007CE0B179B1FDB1937F007E050F
:102C5000B182B1EF75D937D106B1937F01B173B1AC
:102C6000FDB1937F007E06B182B1EF75D93FD10FE0
:102C7000B1917F02B173B1FDB1937F007E07B18244
:102C8000B1EF75D947D106B1937F027E007D007CFC
:102C9000F1B179B1FDB1937F007E08B182B1EF75DA
:102CA000D94FD106B1937FF07EFF7DFF7CFFB179D4
:102CB000B1FDB1937F007E09B182B1EF75D957D1D3
:102CC00006B1937F027E007D007CF4B179B1FDB145
:102CD000937F007E0AB182B1EF75D95FD10FB191B8
:102CE0007F04B173B1FDB1937F007E0BB182B1EF70
:102CF00075D967D106B1937F03B173B1FDB1937FED
:102D0000007E0CB182B1EF75D96FD10FB1917F0107
:102D10007E007D007CF4B1797FFF7EFF7DFF7C1F0C
:102D2000B1937F007E0DB1827F007E007D007C0824
:102D3000B14C75DA0075D980E4F5D8E5D820E1FB0F
:102D400053DBBE75D811E5D820E1FB2290F0AC1220
:102D5000272F90F0AFE0F5DB90F0AEE0F5DC90F0DF
:102D6000ADE0F5DD90F0ACE0F5DE75D8F1E5D8200A
:102D7000E1FB227E007D007CF5B14C75D8087F0018
:102D80007E007D007C00B14C75D8087F007E007D00
:102D9000007C00B14C75D80822B14C75DC01E5DC33
:102DA00030E00553D8FE80F62275B20375800875B1
:102DB000B2017580FE7586EFE4F5B275860D7580FB
:102DC0000C75B2017590FF7591AFF5B275915075A4
:102DD000B20375B03C75B20175B0FF75B17CF5B248
:102DE00075B13C75B03C75B20175C908F5B2227F6A
:102DF000007E007D007C08B14C75DA04227FFF7EE6
:102E0000FF7DFF7C3F227F007E007DA87C0E227F1D
:102E1000007E007DA022E4F5DBF5DC75D83522D1FB
:102E20003D75BCDB43BB0443BB03538FFE75BF0141
:102E300075BBABF5BF22D13D53BBFB80ED75BF0128
:102E400075BB9BE4F5BF438F012290F090743FF077
:102E5000C2AFE5D820E1FBC0D9C0DAC0DBC0DCC01E
:102E6000DDC0DE75BF80D1BDE4F5D8E5D820E1FB3B
:102E700090F08EE5DBF0A3E5DCF090F08EE030E53D
:102E800002718190F08EE0FF5407600690F090741C
:102E900038F0D1BD90F090E05FF4F5DB90F08FE07A
:102EA000F4F5DC75D831E5D820E1FB75BFC0D0DE84
:102EB000D0DDD0DCD0DBD0DAD0D9D2AF2275DA00C9
:102EC00075D981227F05123883EF7002E179F1D440
:102ED0007F05F1DB90F0A5F090F099E090F0A4F080
:102EE00090F09AE090F0A3F090F09BE090F0A2F0C8
:102EF00090F09CE090F0A9F090F09DE090F0A8F0A8
:102F000090F09EE090F0A7F090F09FE090F0A6F097
:102F10007F0512384DC2AFC2C2D13690F0A2E06434
:102F2000AA700FA3E064AA70097D017F551239973A
:102F3000807990F0A2E06433703FA3E0643370398D
:102F4000F5BFF5BCFD7C03FFFE7112F17AE4FFEFE3
:102F5000C3942074809480500974802FF8E4F60F95
:102F600080ED7880761175836FE4F5827F80713F04
:102F7000F17A7D047F5512399722538FFEE4F5BF15
:102F8000FFEFC39432748094805020E4FEEEF1C8C9
:102F90005016E4FDEDF1C8500CE5BC30E20453BC22
:102FA000FB220D80EF0E80E50F80D675BF0175BB4B
:102FB0009B438F0143BB0475BCFF43BB03538FFE90
:102FC00075BBABE4F5BF80FEC394FF748094802290
:102FD00043A820227B017AF0798E221233F490F0FC
:102FE00098E02275C43075C5F875C23075C3F8E431
:102FF000F5C1D2C222C0E0C0F0C083C082C0D0758B
:10300000D00063A201C083C08263A201C000C001DE
:10301000C002C003C004C005C006C00790F0DB7446
:103020003FF0E5D820E1FBC0D9C0DAC0DBC0DCC08E
:10303000DDC0DE75BF8030C704C2C711C1E5B6541C
:1030400001604A53B6FE122EBD75D800E5D820E1C6
:10305000FBAFDBAEDCEF30E51B30E70A90F05C74D1
:1030600080F0EF547FFFEF30E60A90F05C7440F0A0
:10307000EF54BFFF122EBD90F0DBE05FF4F5DBAF45
:1030800006EEF4F5DC75D831E5D820E1FB75BFC05C
:10309000D0DED0DDD0DCD0DBD0DAD0D9D007D0067E
:1030A000D005D004D003D002D001D00063A201D05B
:1030B00082D08363A201D0D0D082D083D0F0D0E080
:1030C0003230002490F03DE004F0700690F03CE0D7
:1030D00004F090F03A11F590F03DE09F90F03CE064
:1030E0009E400CC200E48004E490F03CF0A3F02287
:1030F000EDF090F0AAE0FEA3E0FFC322788E7CF012
:103100007D017BFF7A0079087E007F141229DAE4C2
:1031100090F0A2124276F0A3124276F07F0B1238A2
:1031200083EF6051122FD47F0B122FDB90F02CF025
:1031300090F099E090F02BF090F09AE090F02AF067
:1031400090F09BE090F029F090F09CE090F030F04F
:1031500090F09DE090F02FF090F09EE090F02EF037
:1031600090F09FE090F02DF07F0B12384D7B017AAC
:10317000F07929B1B57F0D123883EF600E122FD48C
:103180007F0D71F47F0D12384DD2037F0712388303
:10319000EF7002416A122FD47F07122FDB90F00BE1
:1031A000F090F099E090F00AF090F09AE090F00939
:1031B000F090F09BE090F008F090F09CE090F00F21
:1031C000F090F09DE090F00EF090F09EE090F00D09
:1031D000F090F09FE090F00CF07F0712384D90F0E7
:1031E00018E004F090F00CE090F046F090F0091236
:1031F00042CC90F008124248D31226C25003124229
:10320000E11242B21242397D3C12428190F04312E7
:10321000422B12427F90F04111F0941EEE940090E8
:10322000F0404005741EF08002EFF090F00B124267
:10323000CC90F00A124248C31226C250031242E157
:103240001242B21242397D3C12428190F050124239
:103250002B12427F90F04E11F0941EEE940090F0ED
:103260004D4005741EF08002EFF07B017AF0793159
:10327000123A843000026147D2007B017AF0792152
:10328000719E7F09716A90F0EAEFF07F0A716A908F
:10329000F0E8716690F0E7716690F0EBEFF07F0C6C
:1032A000716A90F0E9EFF012401E90F07DE0FF901F
:1032B000F018E06F7039C20290F06EE04401F0E067
:1032C0004402F090F06DE04440F0E04480F0A3E070
:1032D0004404F0E04410F0E04420F0E04408F03012
:1032E00003177B017AF0796D7F0A123A02800AD2C5
:1032F0000290F018E090F07DF01240EEA2B6E433B8
:1033000054011242A954FEFDEC124269A295B3E4A5
:1033100033540125E0FFE433FE1242AA54FD124269
:1033200066A202E4FE3354017802C333CE33CED812
:10333000F91242A954FB12426630030B7B017AF06A
:1033400079E67F0C123A0290F05CE0FF6440600581
:10335000EF6480701090F05CE090F053F0122B81DD
:10336000E490F05CF022EFF07F0BAD07123F11AF5D
:1033700005F1CF123F427FA3F1CF123F5FC204128B
:1033800041F3C205719300D205123F0C000000000A
:1033900000D205E4F5B2438608A2059283227F0895
:1033A000716AF1DBEF1225F67F07716AEF541FFF98
:1033B000F1DB900001EF1226087F051242D7900042
:1033C00002EF1226087F041242D7900003EF122664
:1033D000087F06716AEF54079000041226087F03E5
:1033E000F1D5900005EF1226087F02F1D590000676
:1033F000EF022608123B5AE5D820E1FBC0D9C0DA1B
:10340000C0DBC0DCC0DDC0DE1242922400123843B3
:10341000E4F5D8E5D820E1FBB1A9E5DE1225F612E6
:1034200042922404123843E4F5D8E5D820E1FBB1F8
:10343000A990000DE5DB12260890000CE5DC1226B1
:103440000890000BE5DD12260890000AE5DE122642
:103450000875D804E4F5D8E5D820E1FBB1A99000BF
:1034600011E5DB122608900010E5DC12260890001A
:103470000FE5DD12260890000EE5DE12260890F01A
:10348000ACE012383DE4F5D8E5D820E1FBE5DC30CE
:10349000E30F90F0ADF1F424011240CB4408122563
:1034A000F6F1EAE5D820E1FBE5DE30E553B1A9907D
:1034B0000005E5DB122608900004E5DC12260890E2
:1034C0000003124288900002122608123B53F1EAD0
:1034D000E5D820E1FBB1A9900009E5DB12260890B0
:1034E0000008E5DC122608900007124288900006CA
:1034F000122608E924011240CB44041225F6806C00
:103500001242F6B1A9900005EF12428A900004120F
:103510002608900003E4122608900002E412260810
:103520009000041242BF2404B19B900005EF1225C5
:10353000C3123B53F1EAE5D820E1FB1242F6B1A9F0
:10354000900009EF12428A900008122608900007A6
:10355000E4122608900006E41226089000081242A1
:10356000BF2408B19B900009EF1225C31242922498
:1035700002123843E4F5D8E5D820E1FBB1A9900068
:1035800013E5DD122608900012E5DE122608D0DED3
:10359000D0DDD0DCD0DBD0DAD0D922F9E43AFA128F
:1035A000257D1313543F1225F690F0ADE0FBA3E008
:1035B000FAA3E0F92290F0AF123B60E4A3F078B3F5
:1035C0007CF07D017BFF7A00791CFE7F081229DAEE
:1035D000F1F14A4B7002C1A378B37CF07D0190F009
:1035E000AFB1AE123A7D90F0B3E0FF7B63E4FDD162
:1035F000B3EFF0A3E0FF7B0C0DD1B3EFF0A3E0FF3E
:103600007B1FD1B3EFF0A3E0FF7B171DD1B3EFF029
:10361000A3E0FF7B06D1B3EFF0A3E0FF7B3BD1B388
:10362000EFF0A3E0FFD1B3EFF090F0AFB1AC122513
:103630007DFFD1C4AD077F08F1C1B1AC900001F1AD
:10364000C7541FFD7F07F1C1B1AC900002F1C75410
:103650003FFD7F05F1C1B1AC900003F1C7543FFDC0
:103660007F04F1C1B1AC9000041225965407FD7F90
:1036700006F1C1B1AC900005F1C7547FFD7F03D1C5
:10368000A47F02716AEF548090F0B2F090F0AFB175
:10369000AC900006F1C7547FFF90F0B2E04FFD7F81
:1036A00002D1A422AC07123F11AF04F1CFAF05F154
:1036B000CF6182EFC39D5003AF0522EFD39B400340
:1036C000AF032222EF75F00A84C454F0FEEF75F0C8
:1036D0000A84E5F04EFF2290F0AF123B6078B27C96
:1036E000F07D017BFF7A007924123A7D78BA7CF074
:1036F0007D017BFF7A00792C123A7DE490F0C2F0D4
:10370000FCF1F14A4B601690F0AFA3A3E0F9123B35
:103710004D700D123B477008123B4170037F012230
:103720007B017AF079B2719E90F0AFB1AC123B4D53
:10373000FF90F0B7E02F90F0BFF0E0C3943C7480AE
:103740009480400AE024C4F090F0C27401F0123B6F
:1037500047FF90F0B5E02FFF90F0C2E02F90F0BD52
:10376000F0E0C39418748094804006E024E8F07C74
:1037700001123B41FF90F0B4E02F2C90F0BCF0E040
:10378000C3941F748094804003741FF0E490F0BED3
:10379000F090F0BC1242EC7F0BD1A4A31242EC7F5C
:1037A0000AD1A47D807F0CD1A490F0BFE0FFD1C4EA
:1037B000EF547FFD7F09D1A47D027F01D1A47F005A
:1037C00022D1A490F0AF22122596FFD1C4EF22128D
:1037D0003EDF023F17716AEF547FFFEFC4540F754D
:1037E000F00AA4FEEF540F2EFF2275D808E4F5D896
:1037F0002290F0AFE0FBA3E0FAA3E022E4FDE5D8DD
:1038000020E1FBC0D9C0DAC0DBC0DCC0DDC0DE1106
:103810003CE4F5D8E5D820E1FBE5DC5401700EF579
:10382000DC75DB20117BE5D820E1FB7D01D0DED00B
:10383000DDD0DCD0DBD0DAD0D9AF0522EF75F008CF
:10384000A42407FFE5F03404F5DA8FD922E5D82067
:10385000E1FBC0D9C0DAC0DBC0DCC0DDC0DE113C9A
:1038600075DC0075DB08E4117BE5D820E1FBD0DED8
:10387000D0DDD0DCD0DBD0DAD0D922F5DEF5DD75B5
:10388000D8F122E4FDE5D820E1FBC0D9C0DAC0DBE5
:10389000C0DCC0DDC0DE113CE4F5D8E5D820E1FB9A
:1038A000E5DB30E3027D01D0DED0DDD0DCD0DBD043
:1038B000DAD0D9AF052290F0B8EFF0A312273B0081
:1038C000000000E47F707E17FDFC90F0B9F1E3C3C7
:1038D0001226D8502A90F0B8E0FF1237FCEF701F84
:1038E00012429B90F0B9E0FCA3F1D22401FFE43E28
:1038F000FEE43DFDE43CFC90F0B912272F80C42289
:103900003003127F0611B67B017AF079007F063111
:10391000167F0631CF22E5D820E1FBC0D9C0DAC03E
:10392000DBC0DCC0DDC0DE113CE4F5DCF5DBF5DE40
:1039300075DD0875D8F1E5D820E1FB715375D8081D
:10394000317FE5D820E1FB75D804740429F9E43A05
:10395000FA317FE5D820E1FB75D80475D80475DC11
:103960000075DB4075DE0075DD2075D8F1E5D820E7
:10397000E1FBD0DED0DDD0DCD0DBD0DAD0D9221232
:10398000270FE48EDC8FDB12270F78101226E98ECA
:10399000DE8FDD75D8F12290F0AAEFF0A3EDF0787C
:1039A000AC7CF07D017BFF7A007934517D90F0AAE8
:1039B000E090F0AFF090F0ABE090F0AEF07B017AE9
:1039C000F079AC7F0931167F0931CF7F0901B6E567
:1039D000D820E1FBC0D9C0DAC0DBC0DCC0DDC0DE6E
:1039E000113CE4F5DCF5DB75DE0775DD2075D8F1FB
:1039F000E5D820E1FBD0DED0DDD0DCD0DBD0DAD0E2
:103A0000D922715A78B07CF07D017BFF7A00790071
:103A1000517D1235A912257D90F0B2F0900001126F
:103A2000259690F0B3F0714190F0B0F0714790F0AE
:103A3000B1F090000412259690F0B6F0714D90F020
:103A4000B7F090000612259690F0B4F0900007129F
:103A5000259690F0B5F090F0ACE0FF11B690F0AC88
:103A6000E0FF7B017AF079B0311690F0ACE0FF21F5
:103A7000CF78197CF07D017B017AF0794B7E007F55
:103A8000080229DA90F0AC716090F0AC1235AC12FB
:103A9000257D14601E14606B2402600261393002BF
:103AA00009713A1236D75171802D90F0AC1235ACB5
:103AB000E4613612421E5002804F78197CF07D017D
:103AC000713A7E007F081228EAEF3395E04F6011CB
:103AD0005171713A1236D790F0AC1235AC74018046
:103AE0005590F046E0FF64016005EF6402700A90B3
:103AF000F0AC1235AC7402803D90F0AC1235AC7471
:103B000001803390F046E070257B017AF079541201
:103B100035B57B017AF0793E1236D7C280D296C293
:103B20009490F0AC1235ACE41225F602400A90F005
:103B3000AC1235AC74021225F6227B017AF0794B77
:103B4000229000020225969000030225969000051F
:103B500002259675D80875D8082290F0ACEFF0A32E
:103B6000EBF0A3EAF0A3E9F02290F09C7160B15071
:103B7000EF7002FF227FCC71A47F4ED18290F09C27
:103B8000D19B12257DFF71A490F0A0E004F0700697
:103B900090F09FE004F0C390F0A0E09403F1DA40CD
:103BA000DC7F0122AC07E4FBEBB1FA5014A803EC74
:103BB000088003A2E713D8FB5401FAFF71C20B80FF
:103BC000E722AD07D1797F02FE71E6AF05EF3395AD
:103BD000E0FEEF64014E7002D2B57F197E0071E6FF
:103BE000D2B57F057E00D3EF9400EE94004009002B
:103BF00000EF1F70011E80EE2290F08E7160E4A332
:103C0000F078937CF07D017BFF7A00793CFE7F05A4
:103C10001229DAE490F0D8F0A3F0A3F0B150EF70DD
:103C200003FEFF227FF071A4E490F092F090F092F6
:103C3000E0B1FA400281FFE4FAEAB1FA400281C938
:103C4000D1BBEF5403FF90F0D8E0FEC313F0EF6454
:103C5000027007FFB131E4F0806CEF64017007B1CE
:103C6000287401F08060EF6002A12490F092E0756A
:103C7000F008A42A04FC90F091E0F9B18AE0FBEC92
:103C8000D39B4012E4FFB131E4F090F091E004F0F6
:103C9000B18AECF08030ECC39B5017B133E0FF5495
:103CA00001C43333335480FE90F0D8E04EF071C23B
:103CB0008014749329B18CE06C700BB1287401F0FE
:103CC00090F091E014F00A813990F0D8F1D27803A5
:103CD000C333CE33CED8F9FF90F08E1237F42FF9DC
:103CE000EA3EFA90F092E07E0029F9EE3AFAED12FF
:103CF00025F6E490F0D8F090F092E004F0812D9059
:103D0000F0DAE004F0700690F0D9E004F090F09161
:103D1000E0B18AE0600ED171C39405EE64809480B6
:103D20005002811CD171FF2290F0D8E04480F07FD6
:103D30000171C290F092E075F008A42AF582E43592
:103D4000F0F583E5822498F582E58334F0F583224B
:103D5000E4FDFCD17A7FF0D18C7F28D13DFBEB6074
:103D600019C3ED9411EC64809480500E7F057E00A1
:103D7000D13EFB0DBD00010C80E47FC87E0071E6E2
:103D8000AF03EB7F0160027F00222493F582E434CD
:103D9000F0F5832290F0C37160A3EDF0B150EF70A5
:103DA00002FF227F5571A4E4F9E9B1FA502290F0A4
:103DB000C6E075F008A424EEF582E434F0F583E55E
:103DC0008229F582E43583F583E0FF71A40980D967
:103DD0007FBE71A4E490F0C7F090F0C7E0C39409EF
:103DE000748094805010D159D198EF1225F690F03C
:103DF000C7E004F080E37F0122EEC394087480944E
:103E0000802290F09C7160B150EF7002FF227FCC55
:103E100071A47FBED182D15990F09CD19BEF122525
:103E2000F690F0A0E004F0700690F09FE004F0C37C
:103E300090F0A0E09409F1DA40DC7F0122FE71E607
:103E4000A2B5E43322D1797F01D18C7F03D13DFD2E
:103E50007F1B7E0071E6AF0522E4FCFBEBB1FA505C
:103E60000DD1D88002C333D8FC4CFC0B80EEAF04DC
:103E70002290F0D9E0FEA3E022E4F5B243B120C2E3
:103E8000B52271A4E490F09FF0A3F022FE71E6D277
:103E9000B5E4F5B253B1DF2290F0C3E0FBA3E475C3
:103EA000F00112267FA9F0FA22B150EF7002FF2232
:103EB0007FCC71A47F4471A47F0122E4FCFBEBC39F
:103EC000940274809480500DD1D88002C333D8FC02
:103ED0004CFC0B80E9AF0422D145A803EF0822E493
:103EE000FEB1F95026EF30E704D2058002C2051278
:103EF00033930000000000D205F10CEF25E0FF0035
:103F000000000000C205F10C0E80D622A2059282AC
:103F100022F1427FA2D1DFD20512339300000000CC
:103F200000D205F10CE4F5B25386F7000000000062
:103F3000308309C205F10C123382C322C205F10C91
:103F4000D322D20512339300D205F10C00000000F9
:103F500000C2051233930000000000C20580ADE4EA
:103F6000F5B25386F7FEB1F9501FD205F10C0000EF
:103F7000000000EF25E0FF3083034401FFC205F19C
:103F80000C00000000000E80DD2290F0C37160A3E1
:103F9000EDF0E4FE90F0C6E0FD14F0ED6031D19854
:103FA00012257D90F0C7F0E4FFEFB1FA50E690F0F3
:103FB000C7E0FD6E30E00AEE6418C3134480FE8053
:103FC00004EEC313FEEDC31390F0C7F00F80DAAF19
:103FD0000622E0FDA3E0FEA3E02290F09FE06480D3
:103FE000948022E0F8A3E0F9A3E0FAA3E0FB2275B5
:103FF000BF0175B41375B50275BF03E4F5BBF5BF1A
:1040000043A80175880175B30122C0BF75BF014384
:10401000B40375BB9B43B40475BBABD0BF2290F017
:1040200021E090F003F090F022E090F002F090F0A8
:1040300023E090F001F090F024E090F000F090F098
:1040400025E090F007F090F026E090F006F090F078
:1040500027E090F005F090F04DE090F004F0023988
:104060000090F08EEFF0A3EDF090F0997401F0A3C2
:1040700074F0F0A37490F07B017AF0F9123E02EF35
:104080007002FF227B017AF079907D08123F8A90BE
:10409000F098E06F60037F002290F0991237F424CB
:1040A0000611CB54FCFF1225F690F08FE04F12253D
:1040B000F654E3FF1225F690F08EE04F1225F67BC2
:1040C000017AF07994123B697F0122F9E43AFA020D
:1040D000257DAD07AC06EC1224C3E4FBFA798078A9
:1040E00043122421E4FBFA79207842022227E4904B
:1040F000F0B2F0A3F0123EA9EF7002FF227F647EBF
:1041000019123BE6E490F0B0F0A3F090F1161230F3
:10411000F590F0B1E09FEE6480F890F0B0E064803C
:10412000985068E0FCA3E0FD25E0FFEC318EE4F060
:10413000A3F074DC2FF974F03EFA7B01319B90F010
:10414000B1E025E0FF90F0B0E0318EE0FEA3E0FFAB
:1041500011D290F0AC12272FE4FFFE7D207C41901D
:10416000F0AC123FE31223181224FC90F0B2EEF0F0
:10417000A3EFF090F0ECEEF0A3EFF090F0B1E004DC
:10418000F0700690F0B0E004F080807F012233FEF2
:1041900074DC2FF58274F03EF5832290F0B4123B6C
:1041A0006090F0C07401F0A374F0F0A374B7F07BDA
:1041B000017AF0F9123D94EF7002FF227B017AF050
:1041C00079B77D08123F8A90F0BFE06F60037F00EF
:1041D0002290F0C01235AC900001122596FE1225F7
:1041E0007DFDEDFF90F0B41235ACEE8FF012269508
:1041F0007F0122300404C2058002D20512339300ED
:1042000000000000D205123F0C0000000000C205B3
:10421000123F0CD2051233930000000000227F01F0
:1042200012336AEF5408C36001D322EDF090F0A876
:10423000E0FAA3E0FB7C007D18FFAE0212262AA361
:10424000EEF0A3EFF07C0022E02FFFE43E90F0A61A
:10425000F0A3EFF090F0A6E0FEA3E0FFE4FCFD7B0E
:10426000C07AA8F9F822FDEC4EFEED4FFF90F0E683
:10427000EEF0A3EFF022F0A3F0A3F0A3F0A3227DD1
:1042800018AF03AE0202262AE5DD122608E5DE5449
:104290001F2290F0ACE075F008A422C2AF438F015A
:1042A00043BB02538FFED2AF22FF90F0E6E0FCA3A7
:1042B000E02290F0A6E0FAA3E0FB7C007D3C221215
:1042C00025965403C4333354C0FFE922E0FFE4FCD5
:1042D000FDFE78080226FC12336AEF543FFF0237D6
:1042E000DB90F0A674A8F0A374C0F022E0FF1236B1
:1042F000C4EF543FFD22E5DD54FC1313543FFF226D
:00000001FF
